:020000040000FA
:02000000652871
:0800080083120B103C30E200F2
:10001000A0010A280B280C28A00B0928E20B0828AD
:10002000861E3B28061E1F283C30E200A00118282F
:1000300019281A28A00B1728E20B16287D288610ED
:100040003C30E200A001242825282628A00B2328E4
:10005000E20B2228861E4A28061E2A283C30E2008F
:10006000A001322833283428A00B3128E20B302895
:100070000B108B17DF28861406103C30E200A0011D
:10008000412842284328A00B4028E20B3F280B10B0
:100090008B179A28861006103C30E200A0015028E9
:1000A00051285228A00B4F28E20B4E28061E562836
:1000B000861E56283C30E200A0015E285F2860289A
:1000C000A00B5D28E20B5C284E2A83169B011C14B2
:1000D0001A088312FF3A0319CD29223084004030D8
:1000E000A10083169B01831283161C141A089B0A15
:1000F00083128000840AA10B7428831603138113D2
:1001000083160313303086000330850083120313F7
:10011000850100309F008316031300309F00831277
:10012000031303308600970112118B150B108B17E8
:100130006300982883160313A0309F0083120313D3
:1001400002309F0086114030A10022308400103020
:10015000E3009F1BA9289F1FAB28E30BA928831648
:100160008615001C861183121030E3009F1BB628F1
:100170009F1FB828E30BB62883168615801C8611AE
:1001800083121030E3009F1BC3289F1FC528E30B79
:10019000C32883168615001D861183121030E300D4
:1001A0009F1BD0289F1FD228E30BD02883168615CB
:1001B000801D86118312840AA10BA728A328831609
:1001C0000313A0309F008312031302309F00831695
:1001D0000313851083120313861183160313123041
:1001E000920083120313093095000C30970012150A
:1001F0003C30E200A001FC28FD28FE28A00BFB28D3
:10020000E20BFA281F1F02291F1B04293C30A00003
:10021000A00B0829223084004030A10000101F1BD1
:100220000014061006146230A000A00B152918292E
:1002300080101F1B8014061006146230A000A00B53
:100240001F29222900111F1B0015061006146230F9
:10025000A000A00B29292C2980111F1B8015061036
:1002600006146230A000A00B33293629372938291B
:10027000840AA10B0E290330E500223084004030AF
:10028000A10000301F1B01300006E40064180229A1
:1002900000006130A000A00B4B294E2900301F1B2D
:1002A00002300006E400E418022900006130A000DA
:1002B000A00B58295B2900301F1B04300006E40006
:1002C0006419022900006130A000A00B652968298B
:1002D00000301F1B08300006E400E419022900006A
:1002E0006130A000A00B7229752976297729840A2C
:1002F000A10B4129E50B3D29223084004030A100AB
:1003000000080F39E40000306406031902290130A7
:10031000640603190229073064060319022908300C
:100320006406031902290E306406031902290F30EE
:10033000640603190229A10B802986140530A10047
:1003400006103C30E200A001A529A629A729A00B90
:10035000A429E20BA3293C30E200A001AF29B02977
:10036000B129A00BAE29E20BAD2906143C30E20006
:10037000A001BA29BB29BC29A00BB929E20BB829D5
:100380003C30E200A001C429C529C629A00BC3291D
:10039000E20BC229A10BA0297D280330A200033063
:1003A000A3000330A4000330A5000330A6000B30E7
:1003B000A7000A30A8000A30A9000A30AA000230BB
:1003C000AB000530AC000530AD000530AE000D309F
:1003D000AF000C30B0000C30B1000C30B200043073
:1003E000B3000330B4000B30B5000A30B60004305F
:1003F000B7000D30B8000430B9000530BA00053040
:10040000BB000530BC000D30BD000A30BE000A3014
:10041000BF000A30C0000A30C1000430C2000530FD
:10042000C3000530C4000530C5000D30C6000A30D9
:10043000C7000A30C8000A30C9000A30CA000A30B2
:10044000CB000C30CC000C30CD000230CE000D3093
:10045000CF000C30D0000C30D1000430D20003307B
:10046000D3000D30D4000430D5000530D60005305F
:10047000D7000530D8000D30D9000A30DA000A3034
:10048000DB000A30DC000A30DD000430DE0005301D
:10049000DF000530E0000530E1007D284030A1009C
:1004A0002230840083169B018312000883169A0071
:1004B0001C1555309D00AA309D009C149C185E2A86
:1004C0009B0A8312840AA10B552A83161C118312DE
:0204D0007D2885
:02400E00223F4F
:00000001FF
